:020000001829BD
:08000800FF0003088301FE0064
:100010003629A101A117B400FE30872034088728B3
:10002000A0112408031D1728A0150A30A4003808C1
:10003000A8003708A7003608A6003508A500A301C8
:10004000B001AF01AE010A30AD009A20A30A230827
:100050002402031D20282D08031DA011A01D3228F5
:10006000240B35282D08303E8720A40B172814298F
:10007000B200861106118316861106110F3086050F
:1000800083123208A01862283E30A60080308B20F0
:100090003330B10076201330A60088308B207620D4
:1000A00064308A20762064308A202230B1007620A5
:1000B000283061200C30612006306120A014320805
:1000C00062282014B100201C70280611033C031C78
:1000D000752875200730A600D0308B200314080047
:1000E0002014FE3C031985280615201C20108615B7
:1000F0000F3086053108F039860400008611B10EF4
:1001000000002018762832308A2032081429A11BDA
:1001100038280800A601FC3EA500A609031C962865
:10012000FF300000A50703189128A5070000A60FBF
:1001300090280800280830068039B200A81FAB2894
:10014000A509A609A709A809A50A0319A60A03195A
:10015000A70A0319A80AB01FB828AD09AE09AF094C
:10016000B009AD0A0319AE0A0319AF0A0319B00AA0
:10017000A901AA01AB01AC01B901BA01BB01BC01E3
:1001800030082F042E042D040319F6282030B10066
:100190000310A50DA60DA70DA80DB90DBA0DBB0D29
:1001A000BC0D30083C02031DDF282F083B02031D55
:1001B000DF282E083A02031DDF282D083902031C10
:1001C000F0282D08B9022E08031C2E0FBA022F08A2
:1001D000031C2F0FBB023008031C300FBC0203149A
:1001E000A90DAA0DAB0DAC0DB10BC828B21F032988
:1001F000A909AA09AB09AC09A90A0319AA0A031992
:10020000AB0A0319AC0A3908AD003A08AE003B0846
:10021000AF003C08B0002908A5002A08A6002B085A
:10022000A7002C08A80014298313831203130800C5
:10023000A001831681178312FF309F0007308316B9
:10024000850001308600023083129F0089308316BA
:100250009F00CE3083128E00FF308F0090018316F6
:100260000C140C170B178B17831259290C1F4329D9
:100270001F1F3B2910141F1B3E291010CE308E006B
:10028000FF308F000C130C1C54290130BD070301F3
:1002900003180130BE07030103180130BF07030133
:1002A00003180130C0070C107E088300FF0E7F0E7C
:1002B00009008030A1000920A4014008B8003F08CF
:1002C000B7003E08B6003D08B5001020592967293F
:02400E00223F4F
:00000001FF
